:0400000015EF06F002
:08000800046ED8CF05F0E0CF33
:1000100006F00001E9CF0CF0EACF07F0E1CF08F0DD
:10002000E2CF09F0D9CF0AF0DACF0BF0F3CF12F01C
:10003000F4CF13F0FACF14F0F5CF15F0F6CF16F099
:10004000F7CF17F000C00EF001C00FF002C010F0A3
:1000500003C011F09DAA30EF00F09EBA75EF00F0DA
:1000600076A036EF00F077B0F3EF00F076A23CEF29
:1000700000F077B2EFEF00F09DA042EF00F09EB0ED
:100080009DEF00F076AA48EF00F077BAE9EF00F0B4
:1000900076AE4EEF00F077BEE6EF00F00EC000F057
:1000A0000FC001F010C002F011C003F00CC0E9FF56
:1000B00007C0EAFF078E08C0E1FF09C0E2FF0AC0DF
:1000C000D9FF0BC0DAFF12C0F3FF13C0F4FF14C056
:1000D000FAFF15C0F5FF16C0F6FF17C0F7FF045072
:1000E00006C0E0FF05C0D8FF10009EAAFED7AECF25
:1000F00001F1010120A006D0013D03D0466A476A04
:10010000209005D0472C03D0070E0125466E47509E
:10011000472A036A480FE96E000E0320EA6E01C108
:10012000EFFF4650475C01E1208247501D0801E285
:10013000476A9E9A00014EEF00F0D80ECF6EF00E87
:10014000CE6E252AD8B4262A275202E128520BE087
:100150002750D8B42806272E06D0285204E1286A52
:10016000960E276E1F86422AD8B4432A43500608AB
:1001700007E2FF0A03E14250D00802E2819C1F8E91
:10018000292AD8B42A2A2A5203E12950450803E231
:100190002A6A296A1F80212A21500908D8B013D061
:1001A000216A222A22500908D8B00DD0226A232AB7
:1001B00023500908D8B007D0236A242A24503B08CA
:1001C000D8B001D0246A9E904EEF00F0779E4EEF9B
:1001D00000F0819C1F8E769A779A4EEF00F01F8C6C
:1001E00077924EEF00F01F8C77904EEF00F0E339DE
:1001F000700B006ED89000361F0E6F1400106F6EDB
:100200006ECF00F0003A0030070BE35DF9E1120019
:10021000C00E0E0143150309436F3F0E4315436F94
:10022000F80E44150209446FC70E44151809446FAF
:10023000449D448FF80E45150109456F459D000109
:10024000BEEF01F0F5C0FCF0F4C0FBF0FA5352E051
:10025000FBC0E9FFFCC0EAFFF6C0EFFFFB51D8B4DA
:10026000FC07FB07FBC0E9FFFCC0EAFFF7C0EFFF9C
:10027000FB51D8B4FC07FB07FBC0E9FFFCC0EAFF59
:10028000F851030BEF6EFBC0E9FFFCC0EAFFF8C0BA
:1002900000F0003600360036F80E00160050E00B75
:1002A000EF10EF6EFBC0E9FFFCC0EAFFEF5008095A
:1002B000EF6EFB51D8B4FC07FB07FBC0E9FFFCC0A5
:1002C000EAFFF8C000F0003A0032070E00160050B6
:1002D000070BEF6EFBC0E9FFFCC0EAFFF9C000F0BE
:1002E000003600360036F80E00160050F80BEF10FE
:1002F000EF6E3FD0FBC0E9FFFCC0EAFFEF6AFB51A5
:10030000D8B4FC07FB07FBC0E9FFFCC0EAFFEF6ABB
:10031000FB51D8B4FC07FB07FBC0E9FFFCC0EAFFB8
:10032000F6C000F0003A0036E00E00160050E00B78
:10033000EF6EFB51D8B4FC07FB07FBC0E9FFFCC024
:10034000EAFFF6C000F00032003200321F0E001645
:1003500000501F0BEF6EFBC0E9FFFCC0EAFFF7C0C7
:1003600000F0003A0036E00E00160050E00BEF10EF
:10037000EF6E1200040EE36F3ADF4AD7606A9F0EF9
:100380006014606E608460CF10FF709A70980E0EDB
:10039000F56FFB0EF46FF96BF86BF76BF66BFA6B9E
:1003A00051DF0E0EF56FE30EF46FF96BF86BF76B20
:1003B000F66BFA6B47DF0E0EF56FE70EF46FF96B15
:1003C000F86BF76BF66BFA6B3DDF0E0EF56FF469A9
:1003D000F96BF86BF76BF66BFA6B34DF0E0EF56F9B
:1003E000EB0EF46FF96BF86BF76BF66BFA6B2ADFB9
:1003F0000E0EF56FEF0EF46FF96BF86BF76BF66B93
:10040000FA6B20DF0E0EF56FF30EF46FF96BF86BDD
:10041000F76BF66BFA6B16DF0E0EF56FF70EF46FD7
:10042000F96BF86BF76BF66BFA6B0CDF9350FB0B09
:100430000809936EE36BDBDE4CEF02F0266A256A57
:100440002650E55D04E3FCE1E451255CF9E312008C
:10045000D36A400E9B6E646AF29CF29EF2BEFDD798
:100460009D909D9A769A76927690000E926E3B0EB3
:10047000936E800E946E806A816A826A819C819EEE
:100480003E6A3D6A3C6A280E3B6E3F903F92070EE3
:10049000406E010E416E6ED7070ECD6EAA6AD80E61
:1004A000CF6EF00ECE6E1F6A206A3E6A3D6A3C6ACD
:1004B000280E3B6E436A426A456A446A9D8A9D8063
:1004C00076827680768AC00EF212E56BC80EE46FF3
:1004D000B5DF8288818C818E9BEF06F09EA8FED7C7
:1004E000AD6E8BEF02F0819C20802092466A476AB5
:1004F000E66BE4C0E9FFE5C0EAFFEF50E65D0DE220
:10050000010EE625E425E96E000EE521EA6EEFCF47
:10051000E7F0E751E3D7E62BECD71200E7C0EDF0A8
:10052000E6C0ECF0EA5302E1EB5325E0E9C003F04A
:10053000E8C0E9FFE9C0EAFFEF521DE0EDC0EFF0CF
:10054000EC51EC2BD8B4ED2BEE6FE9C003F0E85181
:10055000E82BD8B4E92BE96E03C0EAFFEFCFF0F047
:10056000EFC0EAFFEEC0E9FFF0C0EFFFEA51D8B4F8
:10057000EB07EA07D7D7EA5302E1EB530FE0EDC0F0
:1005800003F0EC51EC2BD8B4ED2BE96E03C0EAFF7D
:10059000EF6AEA51D8B4EB07EA07EDD7E6C001F0FD
:1005A000E7C002F01200266A256A2650000811E210
:1005B000FF0A03E125502C080CE2442AD8B4452A4E
:1005C000455203E14450050801E21F92000E016EFE
:1005D00030D020A2EAD7483C01D003D0000E016EF3
:1005E00028D0030EE425E96E000EE521EA6EEF50F7
:1005F0004A5C03E0000E016E1CD0818C4A50210839
:1006000016E14B5211E14C520FE11F84A10E676FAE
:10061000E76B680EE66FE96B4D0EE86FEB6B060E4D
:10062000EA6F7CDF6E6B03D0010E016E02D0010E0B
:10063000016E12001F92E56B860EE46F54DFE56BCE
:10064000860EE46FB0DF015203E1000E016E44D06C
:10065000E56B910EE46F47DFE56B910EE46FA3DF6E
:10066000015203E1000E016E37D0E56BA70EE46F77
:100670003ADFE56BA70EE46F96DF015203E1000E4F
:10068000016E2AD0E56BB20EE46F2DDFE56BB20E82
:10069000E46F89DF015203E1000E016E1DD0E56BAE
:1006A0009C0EE46F20DFE56B9C0EE46F7CDF015253
:1006B00003E1000E016E10D0E56BBD0EE46F13DF99
:1006C000E56BBD0EE46F6FDF015203E1000E016EBA
:1006D00003D01F82010E016E12001FA215D0E76B1E
:1006E000670EE66FE96BD30EE86FEB6B070EEA6FF0
:1006F00015DFE76B6E0EE66FE96BD30EE86FEB6B01
:10070000070EEA6F0BDF14D0E76B670EE66FE96B3D
:10071000DB0EE86FEB6B070EEA6F00DFE76B6E0E28
:10072000E66FE96BDB0EE86FEB6B070EEA6FF6DE48
:100730002A6A296A1F801200819E7CDF2A6A296A40
:10074000246A24C023F023C022F022C021F0C5DF98
:10075000030E286EE80E276E1F9E1F9A818E04EFEF
:1007600006F01F96E56BC80EE46FBDDEE56BC80EA4
:10077000E46F19DF015204E0010E016E03D002D0D4
:10078000000E016E09EF06F00F0EF26F660EF16FAC
:100790000F0120B708D0F10E6F1408096F6E000129
:1007A000F36B1BD00F0110B709D0F10E6F140609BF
:1007B0006F6E010E0001F36F10D00F0100B709D06A
:1007C000F10E6F1404096F6E020E0001F36F05D075
:1007D0000F01000E016E3BD00001ED51030B006EC6
:1007E000FC0E60140010606E0F0EF56F640EF46F57
:1007F000E9C0F9F0E8C0F8F0E7C0F7F0E6C0F6F0BD
:10080000EEC0FAF01FDDECC065FF659CEFB1658CB2
:10081000F06BEC51F05D14E2EAC0E9FFEBC0EAFFD7
:10082000EFCFF6F0F2C0EAFFF1C0E9FFF6C0EFFF4C
:10083000F12BD8B4F22BEA2BD8B4EB2BF02BE9D761
:100840006086F10E6F146F6E010E016E0F010001D4
:100850004CEF04F00F0120A704D010A702D000B77E
:100860001CD01F90000E3FB2010E0001E46F000E7D
:100870003FB0010EE56FE96BE86BE76B280EE66FA2
:10088000EB6B670EEA6F40C0ECF041C0EDF0E4C0E6
:10089000EEF0E5C0EFF078D70F0100011200E36B36
:1008A0002A6A296A1F90E56BC80EE46FC7DDC2DEB5
:1008B00014DF1FB0CFDF1FB206D0E32BE3510508D2
:1008C00001E2FF00F0D7286A960E276E0BEF06F0C4
:1008D000F56BF46BF36BF26BF0C0F7F0EFC0F6F072
:1008E000F153D8B489D0F6C0E9FFF7C0EAFFF56B41
:1008F000F46BF36BEFCFF2F0F651D8B4F707F607CD
:10090000F6C0E9FFF7C0EAFFEF50FA6BF96BF86F3A
:10091000006A0050F213F851F313F951F413FA512D
:10092000F513F651D8B4F707F607F6C0E9FFF7C09C
:10093000EAFFEF50FB6BFA6BF96BF86F030EF817D9
:10094000F96BFA6BFB6B006A016A0050F2130150FD
:10095000F313F851F413F951F513F6C0E9FFF7C09A
:10096000EAFFEF50FB6BFA6BF96BF86FE00EF817CC
:10097000F96BFA6BFB6B006AF835016EF935026EA4
:10098000FA35036E01360236033601360236033677
:10099000013602360336013602360336E00E011602
:1009A0000050F2130150F3130250F4130350F513E7
:1009B000F651D8B4F707F607F6C0E9FFF7C0EAFF2B
:1009C000EF50F96BF86F006A016AF835026EF9357D
:1009D000036E02360336023603360236033602361B
:1009E0000336E00E02160050F2130150F3130250CA
:1009F000F4130350F51353D0020EF65F000EF75BAD
:100A0000F6C0E9FFF7C0EAFFEF50FB6BFA6BF96B3A
:100A1000F86FE00EF817F96BFA6BFB6BFB31F56FB3
:100A2000FA31F46FF931F36FF831F26FF533F433D3
:100A3000F333F233F533F433F333F233F533F43382
:100A4000F333F233F533F433F333F233070EF517A0
:100A5000F651D8B4F707F607F6C0E9FFF7C0EAFF8A
:100A6000EF50FB6BFA6BF96BF86FF835006EF935E8
:100A7000016EFA35026EFB35036E00360136023622
:100A800003360036013602360336F80E00160050E3
:100A9000F2130150F3130250F4130350F513F2C094
:100AA00000F0F3C001F0F4C002F0F5C003F0A6EFCF
:100AB00005F01F9CE46B320EE36F60AE17D0F10EB1
:100AC0006F146F6E2D98A4902D9071BE2D80719E25
:100AD00060A40BD0000E60B0010E070B006ED89022
:100AE0000036F10E2D1400102D6E1CD00F0110AF2A
:100AF00015D0F10E6F140A096F6E2D88A4922D90F7
:100B000071BC2D80719C1051070B070B006ED890A3
:100B10000036F10E2D1400102D6E03D0000E016E64
:100B20004AD0000165500F0B3A6E2D9A65BC2D8A94
:100B30002D9C62B62D8C000E2DBC010EE86F0F0EA1
:100B4000F06F640EEF6FE8C0F1F0C2D603C031F071
:100B500002C030F001C02FF000C02EF00F0EE76F82
:100B6000660EE66FE56B3A50E55D14E2E6C0E9FF1C
:100B7000E7C0EAFFEFCFEAF0E4C0EAFFE3C0E9FF35
:100B8000EAC0EFFFE32BD8B4E42BE62BD8B4E72B75
:100B9000E52BE9D7F10E6F146F6E2D9EA4BE2D8E3E
:100BA000A49E2DA804D00F01109F03D00001609EC9
:100BB0000F01010E016E015223E0436A426A2E507A
:100BC0000A081EE12F521CE130521AE1315218E19D
:100BD000325053080BE13350590808E134505308A0
:100BE00005E11F8A000179DD0AD00F013250280883
:100BF00007E13350530804E11F8A00016EDD0F0145
:100C000000010FEF06F098D51FA204D01FA601D057
:100C1000A8D501D044D61FB01DDE1FBC4AD71FAED9
:100C200001D0FF00F1D79CEF06F0F86AD09E078E46
:100C30003E0E006E0F0E016E020EE96E000EEA6EA1
:100C4000EE6A002EFDD7012EFBD7A786560EAF6E9B
:100C5000000E7D6EA60EAC6E900EAB6E3E6A3D6AC7
:100C60003C6A280E3B6E3F903F92070E406E030E8B
:100C7000416E0F015C51800B5C6F000E5D6FC19681
:100C8000C198C19A5E6B5F6B34D0020019000012EC
:100C9000008609FF04060001C200A4600006FF01EF
:100CA00097094BB404C000478007FF029207D04663
:100CB0008900000007FF02930005517D0000000835
:100CC000FF039102010142C500000AFF0522000056
:100CD0001300642A8907FF022100FAD61B000000D6
:100CE000C75354532D4F4B00C75354532D4E4700F9
:100CF0000000000EF86E0C0EF76E8A0EF66E0900FC
:100D0000F550006E000A13E00900F550016EE8BED0
:100D100005D00F0BEA6E0900F5CFE9FF01BC090011
:100D200001AC0900F5CFEEFF004EE9D7F9D7F86A1C
:0A0D3000000128EF02F067D703006E
:020000040030CA
:0E00000015127E7C0009910000800FE00F4079
:00000001FF
